:020000040000FA
:1004000021009615632A000020000C08F1008E1AC6
:10041000F1162700131EF11693012000F61430394F
:10042000891A103A7202F202891A0732091E0F3233
:10043000F40374090319F5030A32091E0432F40A9D
:100440000319F50A043210307607031CF600F11A7E
:1004500009007615F61D0900FF30711E0301F40036
:10046000F500F611090023008C0122008C018E0199
:100470002100EF308E00951327003030910092005C
:100480008B1520000C083039891A103AF200F1015E
:10049000F301F401F501F601F6158B170800F108D8
:1004A000031908002000AC1B0800F1018B1373082E
:1004B000B8007408B9007508BA007608BB008B173D
:1004C0000430AD00702B332268224F227722FD3397
:1004D0002100FC3099001A095139031DFC33270013
:1004E00090309B0077233D008E018E1508003D0063
:1004F0001018772B901D08000F088700901120001E
:100500007839031D08000719A7322008343A031D63
:10051000AE328F222000A900090F77329632A00157
:10052000A401A813B01BA8173008C03A03195F3202
:10053000310303194532FC3E031D0232A816003474
:10054000090B2A32330B053283308500C930840011
:100550001234090B053283308500DB3084001934F6
:10056000090B12323230043C0318FF34833085000B
:10057000F4308400B20A0432003F84070318850A6D
:10058000B20BFA33003F0800F43E031DFF34843001
:100590008500B630840039340903090B0732E13095
:1005A0002818E0308400833085000134090BFF34C3
:1005B0003008031D0D323208A8004830AC0000346A
:1005C00030080319FF340030850073308400043490
:1005D000320803190732633A031DFF3421009614D1
:1005E0009611010000308500733084000434310B13
:1005F000053285308500913084002C34090BFF349E
:1006000084308500EF308400A2340508AB00040874
:10061000AA00B708031D043229083602031CA907E3
:100620003D000E122000B01F0932582348305323DA
:10063000240940390838A400A4170800A413A50110
:10064000A908031DF3330C30F2333D000E122000D5
:100650000C301B230C302732A81F02325823E833FA
:10066000A81E0800A81232083D0096000800A81B2A
:100670001732A908031914322B0885002A088400B0
:100680000030870030308600A10803190532A1032D
:1006900016001A00A90BF8330508AB000408AA00DD
:1006A000200940390838A0000830A100A017080030
:1006B000A501A908031908002B0885002A08840051
:1006C0000030870030308600A519053212001E0068
:1006D000A50AA90BF9330508AB000408AA00080015
:1006E00020002C0940390838AC00AC1708003D0048
:1006F000900114309100850120308400F000030146
:100700001A00F00BFD333D000E1796010E120E136A
:10071000901D033290117622FB33163098001E3064
:10072000990020002030A3001030A2002030A70044
:100730001030A6002030AF001830AE002A2B870002
:10074000230015140000000013081A0014081A00F2
:10075000910A0319920A870BF43308002300151637
:1007600015150F322300951615151200930012006F
:10077000940011091F3903190332C123910AF5337B
:10078000951255309600AA3096009514000000008E
:1007900008001234013410340234FF3400340034C1
:1007A0000834D8340434DD34EF34113400340134E7
:1007B000023403340134093402341934003401346E
:1007C00001340034803414340934043400340034E7
:1007D0000134FF34003400340034073405348134EC
:1007E000033408340034323404340334073404341A
:1007F0004E3403345434003455340034203400343F
:100800004334003468340034653400346D340034CB
:100810006E34003469340034743400347A34003473
:100820002C34003420340034453400345734003440
:100830004134003420340034283400345634003439
:10084000453400344234003420340034433400341E
:1008500061340034723400346C3400342034003499
:100860005A3400346534003469340034733400344D
:1008700073340034203400344A3400346534003496
:100880006E3400346134003429340034403403348D
:10089000493400346E3400346B3400347234003424
:1008A000653400346D340034653400346E34003403
:1008B00074340034613400346C34003465340034F2
:1008C0007234003420340034443400347234003440
:1008D00065340034683400346734003465340034DF
:1008E000623400346534003472340034203400340F
:1008F0004934003447340034523400343134003445
:100900003034003430340034303400343034033484
:1009100068340034653400346834003461340034A1
:100920004034003468340034723400347A34003493
:100930002E34003474340034753400342D340034D3
:100940006334003468340034653400346D3400346A
:100950006E34003469340034743400347A34003432
:100960002E340034643400346534003405340F34DC
:100970003934003402341834103405340034383437
:10098000B63408343434A9340934A03447348B34B1
:10099000FD34A034763488341534B63465340034EC
:1009A0000134013401341C34103405340034DF3494
:1009B0006034DD34D83489344534C7344C349C3405
:1009C000D23465349D349E3464348A349F34003488
:1009D000003403340634A2340034023400340A34C0
:1009E0000034003400340034003403340634A234BC
:1009F00000341434003403340034573449344E3452
:100A0000553453344234003400340034003400345C
:100A100000340034003400340034843400340434AE
:100A20000034073400342A3400344434003465344C
:100A3000003476340034693400346334003465346F
:100A40000034493400346E34003474340034653476
:100A5000003472340034663400346134003463345A
:100A6000003465340034473400345534003449349C
:100A700000344434003473340034003400345034CF
:100A800000347B34003439340034373400343534A6
:100A900000344634003434340034343400344434C4
:100AA0000034393400342D340034303400344434CC
:100AB000003430340034383400342D3400343434CD
:100AC00000343334003446340034443400342D349C
:100AD0000034383400344234003433340034453484
:100AE00000342D340034313400343234003437349F
:100AF0000034433400344134003438340034413459
:100B0000003446340034463400344634003439343A
:100B10000034443400347D34003400340034003474
:100B200000342C34033401347734773477342E3462
:100B3000743475342D346334683465346D346E34F4
:100B4000693474347A342E34643465342F347E340A
:100B500068346534683461342F34653477346134F3
:100B60002F344B34723461346D342F34693467342C
:0A0B700072342E34683474346D348E
:00000001FF
